:1000000012C07BC08BC029C028C027C026C025C015
:1000100024C03EC022C021C020C04EC01EC01DC092
:100020001CC01BC01AC011241FBECFE5D4E0DEBF28
:10003000CDBF10E0A0E6B0E0E4E9F4E002C0059036
:100040000D92A036B107D9F710E0A0E6B0E001C0EC
:100050001D92A837B107E1F7E3C1D2CF92E093BF79
:1000600081E089BF83E084BB8EE387BB80E281BBF4
:100070008CE082BBA998C59A87E189B988E58AB9DD
:100080008AE085BF80EC8BBF9093700078940895D0
:100090001F920F920FB60F9211248F9382B78E5238
:1000A00082BF809170008160809370008F910F906B
:1000B0000FBE0F901F9018951F920F920FB60F92C0
:1000C00011248F93EF93FF9380916000882369F050
:1000D0008091600081508093600080916000E82FE3
:1000E000FF27EF58FF4F80818CB9FF91EF918F91DF
:1000F0000F900FBE0F901F9018951F920F920FB682
:100100000F9211248F93809175008F5F80937500FB
:100110008F910F900FBE0F901F9018951F920F9206
:100120000FB60F9211248F93809169008F5F809397
:1001300069008F910F900FBE0F901F9018955D9BD7
:1001400011C080916000882369F080916000815027
:100150008093600080916000E82FFF27EF58FF4FE9
:1001600080818CB95F9BE0C08091700081FFBBC033
:1001700010926C00809170008D7F809370008CB124
:10018000813C41F481E080936A001092600080918C
:100190006B00A7C0823C71F482E080936A0081E02A
:1001A0008093600080916B008CB980916100809396
:1001B0007100BAC0853CA1F481E080936A0082E0BE
:1001C0008093600080916B008CB980916D0090915C
:1001D0006E008093710080916D0090916E0041C01F
:1001E000863CA1F482E080936A0083E08093600003
:1001F00080916B008CB980916D0090916E0080931E
:10020000710080916D0090916E005BC0873CA1F4FD
:1002100082E080936A0083E08093600080916B00AD
:100220008CB98091670090916800809371008091F3
:1002300067009091680045C0893CC1F481E08093DB
:100240006A0082E08093600080916B008CB980919D
:100250007600909177008093710080917600909164
:100260007700892F9927809372005EC08A3CA1F4A1
:1002700082E080936A0083E08093600080916B004D
:100280008CB9809176009091770080937100809175
:1002900076009091770015C08B3CE1F482E080936A
:1002A0006A0083E08093600080916B008CB980913C
:1002B0006500909166008093710080916500909137
:1002C0006600892F99278093720080916100809346
:1002D00073002AC0823D11F48CB921C08034F9F436
:1002E00089E58CB921C080916A00813021F48CB1FC
:1002F0008093620014C080916A00823049F48CB10E
:100300008093620080916A008F5F80936A000CC0C6
:1003100080916A00833041F48CB180936F008091AA
:1003200070008260809370008091700080FFFCCF2D
:10033000809170008E7F809370000895EF92FF92FD
:100340000F931F93CF93182FC62F00E0E02EC39872
:10035000F6DEC39AF4DEA898F2DE57E0F52EC398D5
:10036000EEDE17FF02C0C59A01C0C598110FC7FF86
:1003700002C0C49A01C0C498CC0F000FB0990160AC
:10038000EE0C879B02C081E0E82AD9DEC39AD7DE53
:10039000FA94F7FEE4CFA89AC598A99AD0DEA99856
:1003A000CEDE8E2D9927982F8827800F911DCF9113
:1003B0001F910F91FF90EF900895809175009927FC
:1003C00090937700809376008091690099279093AD
:1003D0006600809365001092750010926900C298C3
:1003E000AEDEC29AACDE0895809175009927909395
:1003F0006E0080936D00809169009927909368004A
:10040000809367001092750010926900C19897DE82
:10041000C19A95DE08955F9BFECF8CB19927089510
:10042000CFE5D4E0DEBFCDBF19DE80E48CB981E436
:100430008CB960916F008091620080DF90936400BE
:1004400080936300809163009091640080936B00BF
:100450008091630090916400892F992780936100B7
:10046000ACDF60916F008091620068DF9093640060
:1004700080936300809163009091640080936B008F
:100480008091630090916400892F99278093610087
:04049000ABDFCFCF40
:00000001FF
